:100000000C942A000C9449000C9447000C9447006F
:100010000C9447000C9447000C9447000C94470044
:100020000C9447000C9447000C9447000C94470034
:100030000C9447000C9447000C9447000C94470024
:100040000C9447000C9447000C9447000C94470014
:100050000C94470011241FBECFE5D8E0DEBFCDBF12
:1000600010E0A0E6B0E0EAECF0E002C005900D92EE
:10007000A036B107D9F710E0A0E6B0E001C01D92AC
:10008000A036B107E1F70E9459000C9463000C946C
:1000900000001F920F920FB60F9211248F93F894C5
:1000A00085B3809585BB8F910F900FBE0F901F90E9
:1000B00018958FEF84BB11BA15BA80E48BBF83E02B
:0A00C00085BF7894FFCFF894FFCFBE
:00000001FF
